:030000000219FDE5
:03000B000200AA46
:03002B0002019936
:03005B0002034F4E
:0300730002033550
:1000800002030406080C10182030406080040608A3
:100090000C10182030406080A0C000070F1F3F0DDB
:1000A0000D0403060D0503030202C2AF306308C24C
:1000B00063857C8AD2AF32C0D0C0E0206227E525BC
:1000C0006002E473E525F4C3334009758A00D26306
:1000D000F57C01D6F58A758B00758D00D262D0E073
:1000E000D0D0D2AF32C3E526334009758A00D2633F
:1000F000F57C01F6F58AC262E526F4603B306803C0
:10010000207213758B00758D00D0E0D0D0C295C2DF
:1001100093C297D2AF32C295C293C297206E0C2081
:1001200066097410D5E0FDE57E4290758B00758DF3
:1001300000D0E0D0D0D2AF32758A00D263757C0097
:10014000C28DD262212B01C4306805206602D2958F
:1001500001C4306805206602D29701C430680520CA
:100160006602D29301C4C29430680A2066077410F4
:10017000D5E0FDD29501C4C29630680A20660774A6
:1001800010D5E0FDD29701C4C29230680A206607FC
:100190007410D5E0FDD29301C4C2AFC2AD53E6EFF7
:1001A000C0D0C0E0D2D3D2AFE57D6009E57A60056A
:1001B000757A00413E757A01C2CEE52A6007207447
:1001C00049152A410A7800790020742EE580307E96
:1001D00001F430E50278FF53DACF207E0343DA20C2
:1001E000307E0343DA10C2D8C271E580307E01F45C
:1001F00030E50279FFC3E89970CB306103752A407E
:10020000207403752A40885FD27020740DE52B603E
:1002100004152B411A43DA01C2D8207002412DA8DF
:100220005F206102C270207402412B88227882B65E
:100230000403852224C3E52594404002D26420CFE4
:100240000AD0E0D0D043E610D2AD32C2CF053AE5B5
:100250007D6009E57B6005757B00612B757B01780E
:1002600002E52A6005307402152AC3E55F94014057
:10027000057562004187756300756C00E5622401B5
:10028000F56250037562FF7982B7020D306D1DC3B0
:10029000E52294324016854D227982B7030E306DE7
:1002A0000BC3E52294324004798E8722C3E523955F
:1002B0002260084004152341BB0523D8CA056CE51C
:1002C0006C7002156CD56D63756D017805C3E56CB6
:1002D000956E4057C3E56C956F50087801756D03B6
:1002E0000202EFC3E56C957050057801756D01C38E
:1002F000E5659524401E7982B704026120206D14C3
:10030000852465E56C046003856E6C756D0175234D
:100310003C02032BE5652850057565FF6120F565F6
:10032000E5650470067563FF756CFFD0E0D0D043BF
:10033000E610D2AD32C2AFC0D053E67FC260759135
:1003400000855694855795759104D0D0D2AF32C2AE
:10035000AF53E6EFC2ADC0D0C0E0C0F0D2D3D2AF51
:10036000A8FBA9FCE57D6007C3E913F9E813F8C20F
:10037000D830710261C153DACF207E0343DA1030E6
:100380007E0343DA20D271E580307E01F420E5025D
:10039000619888278928A1A653DACF207E0343DA03
:1003A00020307E0343DA10C2D8C271307402A192A9
:1003B0007800E580307E01F430E502A192885FA1EB
:1003C0007A53DACF207E0343DA20307E0343DA10FB
:1003D000C271206102819A53DACF207E0343DA1082
:1003E000307E0343DA20C2D8D271885A895BC3E8D1
:1003F0009558F8E99559F97B007E087A00C3E8948E
:100400008CE994005005755E00818C882178A2E605
:10041000A8216055C3E894C8E994005008E4D2E4E8
:10042000FB7A0A8167C3E89468E994015008E4D232
:10043000E3FB7A0F8167C3E894D0E994025008E4A3
:10044000D2E2FB7A1E8167C3E894A0E994055008C4
:10045000E4D2E1FB7A3C8167C3E89498E9940850C0
:1004600008E4D2E0FB7A787E00C3E8955CFCE9956D
:0F0470005DFD30E70AECF42401FCEDF43400FDEF
:10047F00755E00C3EC9AED9E5003755E01885C8932
:10048F005D855A58855B597802A17AC3E89527F89C
:10049F00E99528F9307C02A15E307B02A15E307AAB
:1004AF0002A15720750281BDE9FDE8FC81DCE9C39B
:1004BF0013F9E813F8307902A157E9C313F9E813D8
:1004CF00F8307802A157E9C313FDE813FC20612C23
:1004DF00C3EC941CED9402400281F3ED701EC3EC4B
:1004EF0094C850180529E52970021529C3E52994E8
:1004FF000A5002A192755F00D270A192E5296002A5
:10050F0015297400207F037896E624FAFEE4340060
:10051F00FFC3EC9EFCED9FFD500678007900A15EB5
:10052F00C3EC94FFED9400400678FF7900A15EECD8
:10053F008575F0A4C5F0A2F733F8790040030205E2
:10054F007A78FF790002057AE9C313F9E813F830D6
:10055F007C0EE9600278FFC3E81338F8E43400F941
:10056F00C3E894FFE99400400278FF885FD27020BF
:10057F006102A192741FF4552F4BF52FC274EB70CB
:10058F0002D274752A40307403752A0A306102A1B1
:10059F00A620740353DAFE207403752B20D0F0D0FD
:1005AF00E0D0D0D2AD43E6103279010205D67903FF
:1005BF000205D6790A0205D6791E0205D67964029C
:1005CF0005D679C80205D67817E4D5E0FDD8FAD953
:1005DF00F6227A147B780205FD7A107B8C0205FDDA
:1005EF007A0D7BB40205FD7A0B7BC80205FD7902FB
:1005FF00B27DE4C296D5E0FDD297D5E0FDC297D586
:10060F00E0FDD296D5E0FDD295E576D5E0FDC29519
:10061F007496D5E0FDD9D9EAF8D5E0FDD8FBDBCE4D
:10062F00C29622C37C007D0075F00005F0EA33FA14
:10063F00EB33FB50F6EB13FBEA13FAC3E9FFE8FECB
:10064F00E89AF8E99BF95004EFF9EEF8B3EC33FCB4
:10065F00ED33FDD5F0DFEDF9ECF822E889F08A20D3
:10066F00D2D4F8A9F07B0030F70B7BFFF42401F80C
:10067F00E9F43400F9E88520F0A4ADF0F8E985201D
:10068F00F0A4AFF0FEED2EF974003FFA7C04C3EA3C
:10069F0013FAE913F9E813F8DCF48BF030F70AE8F2
:1006AF00F42401F8E9F43400F9E889F0C2D4F8A988
:1006BF00F0227882B60403020760C3E55F94194005
:1006CF001EE52D54067018206D3678057994E714C1
:1006DF006007780A1460027812C3E54198401F3012
:1006EF006D09856765756CFF756D01852224E4F5CD
:1006FF0045F546F547F548F549C26D020760D26DDD
:10070F007994E7147013E523F43333F913F8E954AC
:10071F000104F9E854FE020754E714147014E5239A
:10072F00F4333333F913F8E9540304F9E854FC02B2
:10073F00075CE523F433333333F913F8E954070433
:10074F0004F9E854F8C39440F8E99400F98845890E
:10075F004622C3E54113F9E54013F8C3E54598F880
:10076F00E54699F9500CC3E89480E994FF401602CE
:10077F000798C3E8947FE994005003020798787FA5
:10078F007900020798788079FF884A894B22E54AD9
:10079F002547F8E54B3548F9854B20E4300701F440
:1007AF003549FA30E709C3EA94F040150207D6C37A
:1007BF00EA940F50030207D678FF79FF7A0F0207EA
:1007CF00D6780079007AF0C3E5249564500AC37493
:1007DF00019524500B0207F4E54B20E70E0207F4B6
:1007EF00E54B30E706884789488A492278A4E6FA1C
:1007FF00C3E54A33F8E54B33F912066AE930E70BE4
:10080F00C3E89480E994FF4013012FC3E8947FE974
:10081F0094005002012F787F7900012F788079FFA3
:10082F00E820E715C3E52398F84009C3E894014091
:10083F00030208567801020856E8F424012523F82C
:10084F00400302085678FF884C2278A5E6FAA8489C
:10085F00A94912066AE930E70CC3E89401E994FF4D
:0E086F00401602088BC3E894FFE99400500382
:10087D0002088B78FF790002088B780179FFE92057
:10088D00E715C3E54C98F84009C3E894014003020D
:10089D0008B278010208B2E8F42401254CF84003AF
:1008AD000208B278FF88242278FFC26420693D20B7
:1008BD006A12D264C3E541940A4009C3E525944008
:1008CD005002C26479A1E76023E541601F74FF8582
:1008DD0041F0848539F0306A0375F005A4F8C5F050
:1008ED00600278FFC3E895675002A867886622C347
:1008FD00E54094C8E5419400E566500314210D04CC
:10090D006002F566227883E6F520120FCA75E8902D
:10091D001205B875E890E5E820ECFBA8BDA9BE125C
:10092D001064757155757200C3740013FD745560B4
:10093D006613FC74552CFC74003DFDECFAEDFBC305
:10094D00E89AE99B4014E5712455F571E572340080
:10095D00F572EA2CFAEB3DFB80E5AE71AF72C3E5A3
:10096D007213F9E57113F8C3E913F9E813F87A0373
:10097D00C3E913F9E813F8DAF7AA201A70097571AB
:10098D00007572000209A41AEA6008EE28FEEF391C
:10099D00FFDAF88E718F722275E890227883E6FF68
:1009AD00E5E820ECF7A8BDA9BE0573C3E57394086F
:1009BD004052757300E9FA79A0E76044EA7007E5E3
:1009CD0074601B0209DFC3E895746010E57450066E
:1009DD00600C140209EB0460F90209EBE574F5747F
:1009ED00C39472401B7564C0C39404401375648036
:1009FD00C39404400B756440C394044003756400B4
:100A0D0075BB0822EFC39401601F7455601BC3E8CA
:100A1D0094FFE994035012C3E89571E9957250095A
:100A2D00E564600C1564020A3DE564F4600205643A
:100A3D00A864C3E524985002A824C3E89565400A2C
:100A4D00A865E565F4600385656488258826E573EA
:100A5D00B4070375BB1022743279A687F0A4C5F0D4
:100A6D00A2F733F8C3E895644002A864882288246D
:100A7D00882588268867227540007541F022C2AF0F
:100A8D0075C820A8CCA9CDAA3A30CF010A75C824C3
:100A9D00D2AFC3EA13FAE913F9E813F8AB3BAC3C58
:100AAD00883B893CC3E89BF8E99C20690A547FF98F
:100ABD0030670261AE610BAD3D8A3DF9EA9D547F11
:100ACD00FA600478FF79FFAE3EAF3F8B3E8C3FC39B
:100ADD00EC9FFCC3E99CF542A83BA93CC3E89EF8FA
:100AED00E99FF9C3E54113FBE54013FAE82AF54008
:100AFD00E93BF54150067540FF7541FF6155AA4030
:100B0D00AB41AC40AD417E047F02C3EB9404400287
:100B1D001E1FC3EB940840021E1FC3ED13FDEC1303
:100B2D00FCDEF7C3EA9CFAEB9DFBEF6009C3E9130A
:100B3D00F9E813F8DFF7EA28FAEB39FB8A408B4125
:100B4D0050067BFF8B408B41C3EB94025002D26762
:100B5D003069047F0361807892E6FFC3E5379482A4
:100B6D0040110FC3E53794A040010FC3EF94064029
:100B7D00027F057E03E541C4540FF9E541C454F0ED
:100B8D00F8E540C4540F28F8C3E89EFAE99400FB39
:100B9D004009C3EA9402EB940050047A02E4FB612D
:100BAD00FAAA40AB41EBC4FEEAC4540F4EFCC3EAB3
:100BBD009CFAEB9400FBC3E813C313F8EA28FAEB95
:100BCD003400FB8A408B41C3EB94024002C267782C
:100BDD0003EBC4FE7B00EAC4540F4EFAC3EA98FA45
:100BED004005C3940250027A027892E6FF3060020B
:100BFD0061FA855256855357D26043E680C3E49A15
:100C0D00F8E49BF9C3E833F8E933F9306702819BC7
:100C1D00E8FAE9FBD3E913FDE813FC88528953C3C5
:100C2D00EF94036038EF20E00DE82CF8E93DF9EC86
:100C3D00FAEDFB020C56E828F8E939F9C3E824026D
:100C4D00F8E93400F97AFE7BFFC3EF9403400E8A76
:100C5D00548B55884E894F8C508D5181CF88548936
:0F0C6D00558A4E8B4F8C508D51306920C3E53323
:100C7C0094034019E542A2E713F8E555F424013832
:100C8C00400B20E7087554FFF42401F55581CFE89B
:100C9C00FAD3E813FC8852C3EF94036020EF20E0F2
:100CAC0007E82CF8ECFA81BBE8282402F87AFEC39A
:100CBC00EF940340088A54884E8C5081CF88548A14
:100CCC004E8C50E56BC3335002646BF56B30600295
:100CDC0081D9753404D26043E680E52D5406601F3B
:100CEC00A840A941C2AF53E67F759100C3E498F5C3
:100CFC0094E499F595759104D26043E680D2AF22C5
:100D0C00D265754400752000306B03752040020DD0
:100D1C002BD265754400752040306B03752000D2D2
:100D2C00AF7801206722E52D54066002C265C3E549
:100D3C0041940540137802940540087803940540CB
:100D4C00027806306902780A206019E54460153093
:100D5C00690AC3E53394034003D53406D2AFD26C91
:100D6C00C10D91E1D2AF0000C2AF20672AE541C3AB
:100D7C00FB940F40027B0FEB240530730123306A88
:100D8C0002742820620123F93069027982E58D13FF
:100D9C00E58B13C39940B10544E59B5440B5200243
:100DAC00A1F730690A08C3E8940A400108A154204D
:100DBC006502A12BC26553E67F75910030671075F3
:100DCC0094007595FC759104D26043E680A12BAE1E
:100DDC0040AF41C3EE33FEEF33FF50047EFF7FFF85
:100DEC00C3E49EF594E49FF595A1D1C3E533940239
:100DFC005002A12B306502A12BD802C10BA154C209
:100E0C006C53E67F759100855494855595759104C6
:100E1C00854E56854F57D26043E680D2AFE52D54B0
:100E2C00066008206A020533020E47306C0D206BF9
:100E3C000A206507158115810216A92278003064F5
:100E4C00053065027801E53775F007A4F9E5F0285F
:100E5C00F5F0E9A2F013A2F113A2F213F537C39443
:100E6C00785003753778C3E53795384008D266C299
:100E7C0095C293C297306002C181855056855157F7
:100E8C00D26043E68022207D11C2AF754302C29628
:100E9C00D294D2AF759F11021061C2AF754302C2DA
:100EAC0096D292D2AF759F11021061307243207DA1
:100EBC0020C2AF754303900177757E40C293C292F6
:100ECC00306204D297C1D5D296D2AF759F1302105F
:100EDC0061C2AF754303900177757E40C295C29491
:100EEC00306204D297C1F5D296D2AF759F10021022
:100EFC0061207D17C2AF754303900152C2933062DB
:100F0C0002D297D2AF759F13021061C2AF75430323
:100F1C00900152C295306202D297D2AF759F1002E7
:100F2C001061207D11C2AF754304C294D292D2AF2E
:100F3C00759F10021061C2AF754304C292D294D255
:100F4C00AF759F13021061307243207D20C2AF75C4
:100F5C004305900166757E10C297C296306204D22A
:100F6C0095E171D294D2AF759F11021061C2AF7529
:100F7C004305900188757E04C297C296306204D2F4
:100F8C0093E191D292D2AF759F11021061207D171F
:100F9C00C2AF754305900148C297306202D295D218
:100FAC00AF759F11021061C2AF75430590015CC211
:100FBC00973062EBD293D2AF759F11021061207DF6
:100FCC0011C2AF754306C292D296D2AF759F13026F
:100FDC001061C2AF754306C294D296D2AF759F1002
:100FEC00021061307242207D20C2AF754301900126
:100FFC0088757E04C295C294306204D293010DD2DE
:10100C0092D2AF759F10021061C2AF75430190016F
:10101C0066757E10C293C292306204D295012DD2B5
:10102C0094D2AF759F130161207D16C2AF75430139
:10103C0090015CC295306202D293D2AF759F1001C1
:10104C0061C2AF754301900148C293306202D295E0
:10105C00D2AF759F13C26622900146757E00C29571
:0F106C00C293C297C294C292C296C26222788087
:10107B0076070876070876010876040876FF087667
:10108B00FF08760A087602087601087601788C76D6
:10109B00010876000876B40876FF0876FF0876FF1D
:1010AB000876030876FF0876010876FF0876250890
:1010BB0076D00876780876C80876040876FF087626
:1010CB000108760008767A08760A08760108760118
:1010DB000876000876FF227887E6FFC272BF03020C
:1010EB00D2727888C27DE630E102D27DC27E7889E9
:1010FB00E630E102D27EC3EF94026008758E01D216
:10110B0073021114758E00C273227880E61490005E
:10111B00809378A4F67881E6149000809378A5F6F6
:10112B007886E61490008D9378A6F6789FE6F87093
:10113B000108C3E8941140027811E82828F56E25C0
:10114B006E256E28F56F256E2828F570789CE67550
:10115B0038FF75390CB402067538A075390AB4031B
:10116B000675388275390578A3E61490009A93F5C5
:10117B0069116422227896E6FA7897E6FB7888E67E
:10118B00B40305C3EB940EFB307F047A007BFFC3E3
:10119B00EB9AFCC3948250027C827575000575EC4A
:1011AB008575F0A4C3E5F0947D40F222D27F3180A7
:1011BB001205C77A007B007C101205BDE55F2AFA89
:1011CB0074003BFBDCF37C04C3EB13FBEA13FADC8C
:1011DB00F7FEC27F318022E5EF20E6037520000584
:1011EB0020903FFFE520146006901DFF14600093D4
:1011FB0004600375EF1253D9BF7581C043FF801292
:10120B0005B875EF0243B203E5B3240420E70DF5EF
:10121B0021E5E320E0068521B343E30111647580EA
:10122B00FF75A40075F1B275D4DF75900175A5FC3F
:10123B0075F2FE75D50175A60175E241E4F8F6D895
:10124B00FD756B0111791216F87898867675300159
:10125B00C2AF1205D11205E11205C71205E812053E
:10126B00C71205EF1205C712181A1205D11205D1B4
:10127B001205CCC2AF78FA79FA308507D9FBD8F7CB
:10128B00021C0011E23115317F318078988676117E
:10129B006475A90075B680757D00758850758912C7
:1012AB0075C82475910475D84075A82275B8027558
:1012BB00E690759B80759D0075D10E75BCC075BB96
:1012CB000875BA1175E8801205B8D2AF120912531E
:1012DB00DACF207E0343DA20307E0343DA1043DA81
:1012EB0001C2D8C2711205D1D2617B037A0CE55EC3
:1012FB0070077A0CDB0302127E1205C72070030203
:10130B00127EC270E55FC3940240E1E52F541F8546
:10131B006160F561B560D5DAD5C26153DACF207E55
:10132B000343DA20307E0343DA10C2D8C27178A2AD
:10133B00E67008D274E52F54E0F52FC275752900BD
:10134B001205CC307409C3E529940A4002D27512F8
:10135B0005BD78023074027800C3E55F9840F0C297
:10136B00AF1205E11205E11205E1D2AF1205D175FD
:10137B004D001205BD788CE6C39401500302145343
:10138B00E530C394015003021453207435C3E55F59
:10139B0094FF5003021453C2AF1205F6D2AF1205DD
:1013AB00CCC3E55F940150EFC2AF1205E11205C249
:1013BB001205E1D2AF1205CCC3E55F94FF40E90201
:1013CB00189F7F05D27F31801205CCC2AFC27F310F
:1013DB0080AE5FC3E55F947FD2AF40761205B8C293
:1013EB00AF1205F6D2AFDFDC31B7C3EE94057897B9
:1013FB00F61205D11217391218227F0AD27F3180CB
:10140B001205CCC2AFC27F3180AE5FC3E55F947F64
:10141B00D2AF50E61205B8C2AF1205E11205C212E7
:10142B0005E1D2AFDFD631B7EE24057896F612057B
:10143B00D11217391218511205CC3180C3E55F94C4
:10144B00FF5002619502189FC3E55F954D400385E0
:10145B005F4D1205CC78017988E7B403027805C398
:0F146B00E55F984002617DC2AF1205F61205F6EB
:10147A001205F6D2AF1205D1753000E4F531F53216
:10148A000531E531F470390532789AE67819146035
:10149A0012783214600D787D14600878FA146003AB
:1014AA00753200C3E53298401715327531B4789910
:1014BA008676C2AF1205F6D2AF789886761205CC38
:1014CA001205C2E52A7005307402417E7801207443
:1014DA00027806C3E55F9840A71205CCE52A700397
:1014EA0002127EC2AF1164E4F522F523F524F52534
:1014FA00F526F56AD2AF7885E6C333F568E4F54593
:10150A00F546F547F548F549F573F52CF52DF53708
:10151A0075730875BB101205B81209A5E5E820EC29
:10152A00FBA8BDA9BEE97001F888741209A97573F0
:10153A000875BB107887E6FE760211E27887EEF628
:10154A00C2AF7564FF120A6485226485226585220A
:10155A0066D2AF75220175240175250175260185AC
:10156A00636C756D0175B69075A903757D017888F0
:10157A00E6B40307C27D307602D27DD268D269759D
:10158A003300120FCA120FEF120A84120A8B120AC0
:10159A0084120A8B120A840215B0C2AF11E2D2AFCA
:1015AA0075730075BB08120D1D1206C1120E481282
:1015BA000E92120A8B120D0C306D0312076120670E
:1015CA00031208B53067031208FC120E48120EB750
:1015DA00120A8B120D1D306D0312079D120E48124E
:1015EA000F2E120A8B120D0C306D031207FB120E0E
:1015FA0048120F53120A8B120D1D306D031208592F
:10160A00120E48120FCA120A8B1209A5120D0C12D9
:10161A000E48120FEF1209A9120A8B30692F206B9C
:10162A002C85676485676585636C756D0179187AA1
:10163A000CC3E533994009C269D26A8A3502165742
:10164A00C3E55F940140030215B00216B1306A1B6C
:10165A00206B18E535147004C26AA1A4F535C3E5F8
:10166A005F940140030215B00216B1753600C3E556
:10167A00629401400985676585636C756D01C3E5F0
:10168A006278FA985021307404E52A601A78F030AA
:10169A006B058567647820C3E541985002A1B005BF
:1016AA0036E55F6002C1B4753600C2AF116478874F
:1016BA00E6FE760211E27887EEF6E4F522F523F5E6
:1016CA0024F525F526F568C26875A90075B68075F2
:1016DA007D00D2AF1205B81164307406E52A700293
:1016EA00417E788DE6C394014002615A8185901A41
:1016FA000D782012177BE520B4A50CA312177BE501
:10170A0020B45A030217191179121739021738909F
:10171A001A0378807B0A12177BA308DBF9901A0F49
:10172A00788C7B1812177BA308DBF9901A2722C240
:10173A00AF1217BA121794901A00740E121780A3D8
:10174A007404121780A37414121780901A037880F5
:10175A007B0A12177FA308DBF9901A0F788C7B1883
:10176A0012177FA308DBF91217CD1217AB901A27AD
:10177A0022E493F622E6438F01538FFD75EF02753B
:10178A00B7A575B7F1F0538FFE22438F02438F013D
:10179A0075EF0275B7A575B7F1901A0DF0538FFC66
:1017AA0022901A0D74A5F180901A0E745AF18022B3
:1017BA007A3079D07820901A40F17BE520F709A396
:1017CA00DAF7227A3079D0901A40E7F18009A3DA61
:1017DA00F922AB77A878BB01027980BB0202798132
:1017EA00BB03027982BB04027994BB05027983BBED
:1017FA0006027986BB07027992BB08027987BB0980
:10180A0002799CBB0A027988BB0B027989E8F72224
:10181A007C051205D1DCFB22C2AF1205E11205E8F4
:10182A001205EF1205F61205C21205E11205E812B9
:10183A0005EF1205F61205C21205E11205E81205B6
:10184A00EF1205F6D2AF22C2AF1205F61205EF1259
:10185A0005E81205E11205C21205F61205EF120596
:0D186A00E81205E11205C21205F61205EFA5
:101877001205E81205E1D2AF22AE77AF78C2AF12F8
:1018870005E11205E11205E11205C2DEF21205F6C5
:101897001205C2DFF8D2AF221122111A111A757779
:1018A7000175780175790011807C05AD5F1205D14E
:1018B700C3ED955F70F5C3E55F9401400AC3E55F2B
:1018C70094FF40340218DD1217DC1217391122C2B7
:1018D700AF75EF12111ADCD30579C3E5799403507C
:1018E7000280C4111A0578E5771490009F93F808D1
:1018F700C3E57898500280AC111A111A0577C3E531
:1019070077940C5002809A121079121739C2AF756A
:04191700EF12111AA0
:0319FD000211E2F2
:101A00000E041407070104FFFF0A020101A55A0191
:101A100000B4FFFFFF03FF01FF25D078C804FF01DA
:081A200000FF0A010100FFFFB5
:101A4000234656544C6962656532304150726F23AB
:101A500023424C48454C492346333930232020202B
:101A60002020202020202020202020202020202076
:101C0000C2AFC2D353D9BF7581C043B20343FF8073
:101C1000752438752503B1C975EF0275E24043F1AB
:101C20002053A4DF75D400D2857DFA780379E67C51
:101C300010752200752300901DD67B0675249875BB
:101C400025013085028142208508D8FBD9F9DCF7CF
:101C500081B4308508D8FBD9F9DCF781B4B189E4C7
:101C600093A3C39A6004DDC381B4DBDBB17B600264
:101C7000812B7B08E493FAA3B15CDBF87A30B15C8A
:101C8000752200752300B17BEAFCEBFDC3ED94FEE9
:101C9000400EB17B8A278B28ED30E0048A828B834B
:101CA000B17B7AC270D8C3ED94FE601350CEBD00F4
:101CB00025EC60097520007521FF0200008100A855
:101CC00027A9280809D804D90281D3B17FEA89AAB3
:101CD000F281C50D81A0C3ED94035049EDA2E092BD
:101CE000007AC5C3E5829400E583941C50902000DF
:101CF00010438F02438F0175B7A575B7F1F030001F
:101D00001FA827A9280809438F01538FFDD804D99C
:101D100002A12089AAE275B7A575B7F1F0A3A10DBC
:101D2000538FFC817C7AC1BD030CE493A3FAB140CC
:101D3000DCF8B138817C817EAA22AB23B15CEBFA5E
:101D4000EA6222752608C3E52313F523E52213F57D
:101D50002250066323A0632201D526EAB1C9B1C986
:101D600075260AEAF4200102D285300102C285B14B
:101D7000C9C3134002C201D526EB22B17FEAFB2082
:101D80008502A17F308502A184752608AE24AF2587
:101D9000C3EF13FFEE13FEB1CDB1C9C3EA13308513
:101DA000024480FA30E703632201C3E52313F523DD
:101DB000E52213F52250066323A0632201D526D91C
:101DC000E52265236523F52222AE24AF250E0FDE22
:101DD000FEDFFCD20122424C48656C693437316326
:041DE000F390060175
:00000001FF
